:1000000000EEFCF0EE6AEE6AEE6AEE6AF0EF1FF0C8
:103E9000EECF00F0EECF01F0EECF02F0EFCF03F067
:103EA00064EF1FF0036A026A016A006AE950EA10CF
:103EB00008E003C0EDFF02C0EDFF01C0EDFF00C050
:103EC000EFFF000CE96AEA6A0050086E0150096EC3
:103ED00002500A6E03500B6E026A036A0850040215
:103EE000F3CF00F0F4CF01F008500502F3500126A3
:103EF000F450022209500402F3500126F450022229
:103F0000D8B0032A08500602F3500226F4500322C8
:103F100009500502F3500226F45003220A5004020D
:103F2000F3500226F450032208500702F3500326F0
:103F300009500602F35003260A500502F3500326E7
:103F40000B500402F350032656EF1FF0FC00720ED4
:103F5000046E010E056E066A076AFC0EE96E000E1D
:103F6000EA6E48EC1FF00001FF0EFC07FD23FE2364
:103F7000FF23FF51FC11FD11FE11D8B41200F3D73D
:103F8000FC00250E046E056A066A076AFC0EE96EDF
:103F9000000EEA6E48EC1FF00001FF0EFC07FD2347
:103FA000FE23FF23FF51FC11FD11FE11D8B41200B6
:103FB000F3D7949482941200D96E8294D950000160
:103FC000FC6FFD6BFE6BFF6BDCDF8284D950000160
:103FD000FC6FFD6BFE6BFF6BD4D7190E93121200B2
:103FE000F26AE7DFFADF81B602D0010EE5DF81B8C1
:103FF00002D0020EE1DF81B0F6D7030EDDDFF3D78A
:020000040030CA
:0A000000FF32F9FEFFFBBFFFFFFF18
:00000001FF
